:020000040000FA
:100000000A128A11092800008000840AA30B042820
:1000100008008313273084002530A300003004201B
:100020008312A4017528CA01CB012D288312031362
:10003000F230A0000A30A1002830A2000A128A1172
:10004000A20B1E280A128A11A10B1C280A128A115F
:10005000A00B1A28CA0A0319CB0A4A084802A000B2
:100060004B0849022004031D162808008312C6000D
:10007000460883169B001C141A088312C700470801
:100080000800C400450883169A00831244088316AA
:100090009B001C158B138B1355309D00AA309D00BF
:1000A0009C14000000008B171C119C185528080098
:1000B00027308316990018150800582083168C12D3
:1000C0000C129816903083129800080083128C1E30
:1000D0006C281A08C3006E2820107328981C7228F8
:1000E000181218162014430808005D208028A81351
:1000F0002808860083168613080083160617080052
:1001000077207D2044308312A500A60107309F0090
:100110009628C100C2014108C800C90113208312FA
:10012000C20A0A304202031D8B280800831685018B
:100130000614061286120613861383122710270848
:100140008500A71027088500271127088500A7111B
:1001500027088500281228088600A812280886008B
:10016000281328088600A81328088600AA01AB01D6
:100170009030AF008030B000B030B100C629BA0076
:100180003A0836208312BD003D08BA0040303A02DA
:1001900040100319CD28031C40143C082902C0104C
:1001A0000319C01440154018C01C4011401D3629C9
:1001B0003A09BE0001303E05BF003F084012031D52
:1001C00040162710401A2714270885003A09BE0058
:1001D00002303E05BF003F084012031D4016A71025
:1001E000401AA714270885003A09BE0004303E05CE
:1001F000BF003F084012031D40162711401A271563
:100200002708850020303A05BE003E084012031D35
:100210004016A812401AA8162808860010303A0581
:10022000BE003E084012031D40162813401A28172E
:100230002808860008303A05BE003E084012031D1B
:100240004016A813401AA817280886003B0803196F
:100250002D29A715270885003029A7112708850013
:10026000281628088600281228088600080083120D
:10027000AD01B901BB012908BC002D08BF208312C4
:10028000AD0AB90A7F303902031D3A290800B600C9
:10029000B61F5229AB01F0303605AA000F303605E3
:1002A000B7000800AB0A01302B02031D5A2936089B
:1002B000AD00080002302B02031D8E293608AE0067
:1002C0002A0831023811031938157B302D02B81174
:1002D0000319B81538163819B81D3812381E742984
:1002E00037218312AB0108002A083002031D82293E
:1002F000AE012E08BB003708BC002D08BF208312BA
:10030000AB0108002A082F02031D8E292E08BB000E
:100310003708BC002D08BF208312AB010800B500D0
:10032000B51F9A29AB01F0303505AA000F3035050D
:10033000A900080003302B020319A1290318A129E1
:10034000AB0A01302B02031DA8293508AD000800B7
:1003500002302B02031DC5293508AE002A082F02E2
:10036000031DC5292C08031DB9292908C500003023
:10037000412083122E080319C3292C08C5002D081B
:1003800041208312AC0A0330AB0008000130892001
:10039000372183120618EF290130892083120618AD
:1003A000EF29AC01B4017F30C5002C084120831235
:1003B000AC0AB40A7F303402031DD329AC010330E8
:1003C000AB0083120618EF2966208312B2003312A5
:1003D00020183316331EE12932088F21E12901301C
:1003E0008920003036208312A90066208312B200D3
:1003F000B3122018B316B31EF52932084721F52988
:02400E00023D71
:00000001FF
